:020000040800F2
:10000000F84000209D0100089B1000087D0F0008AB
:1000100099100008A9020008D5150008000000008A
:100020000000000000000000000000009F10000819
:10003000AB020008000000009D100008A11000089D
:10004000B7010008B7010008B7010008B7010008B0
:10005000B7010008B7010008B7010008B7010008A0
:10006000B7010008B7010008B7010008B701000890
:10007000B7010008B7010008B7010008B701000880
:10008000B7010008B7010008B7010008B701000870
:10009000B7010008B7010008B7010008B701000860
:1000A000B7010008B7010008B7010008B701000850
:1000B000B7010008B7010008B7010008B701000840
:1000C000B7010008B7010008B7010008B701000830
:1000D000B7010008BD150008C9150008B7010008E0
:1000E000B7010008B7010008B7010008B701000810
:1000F000B7010008B7010008B7010008B701000800
:10010000B7010008B7010008B7010008B7010008EF
:1001100079110008B7010008B7010008B70100080D
:10012000B7010008B7010008B7010008B7010008CF
:10013000B7010008B7010008B7010008B7010008BF
:10014000B7010008B7010008B7010008B7010008AF
:10015000B7010008B7010008B7010008B70100089F
:10016000B7010008B7010008B7010008B70100088F
:10017000B7010008B7010008B7010008000000003F
:10018000B7010008B7010008DFF80CD000F07AF8DA
:100190000048004715160008F84000200648804730
:1001A00006480047FEE7FEE7FEE7FEE7FEE7FEE75C
:1001B000FEE7FEE7FEE7FEE72511000889010008DB
:1001C0002DE9F05F0546002092469B46884606468C
:1001D000814640241BE0284641464746224600F01F
:1001E00041F853465A46C01A914110D31146184659
:1001F000224600F028F82D1A67EB01084F462246E8
:100200000120002100F01FF817EB00094E41201ECD
:10021000A4F10104DFDC484631462A464346BDE8E6
:10022000F09FD2B201E000F8012B491EFBD27047CB
:100230000022F6E710B513460A4604461946FFF7B2
:10024000F0FF204610BD202A04DB203A00FA02F11C
:10025000002070479140C2F1200320FA03F31943B4
:1002600090407047202A04DB203A21FA02F0002156
:10027000704721FA02F3D040C2F1200291400843B6
:1002800019467047064C074D06E0E06840F0010350
:1002900094E8070098471034AC42F6D3FFF778FF94
:1002A000CC160008EC160008FEE77047704790F87F
:1002B0003510022903D080214165012070470521B6
:1002C00080F835100068016821F00101016000200C
:1002D0007047000070B5044600F0ECF80546601C5D
:1002E00002D004480078044400F0E4F8401BA04227
:1002F000FAD370BD240000202DE9F84FDFF87CB15F
:1003000000224FF001084FF0030A4FF00F090BF1E4
:10031000040E00BF0B6808FA02F42340A3426ED11A
:100320004D68022D01D0122D0ED1D50800EB850CA1
:10033000DCF820505607F70E09FA07F6B5430E69A8
:10034000BE402E43CCF82060066855000F790AFAAB
:1003500005FC07F0030726EA0C06AF4037430760A9
:100360004E68012E05D0022E03D0112E01D0122E80
:100370000ED18668CF6826EA0C06AF403743876007
:100380004668A6430C79C4F3001494403443446097
:10039000C6688C6826EA0C06AC403443C4604C68DE
:1003A000E40065D5364C256845F480452560246811
:1003B00022F0030504F480440094324C2E19D6F840
:1003C000084895072F0F09FA07F5AC432E4DA842B0
:1003D00001D1002524E02D4DA84201D101251FE0C7
:1003E0002B4DA84201D102251AE02A4DA84201D185
:1003F000032515E0284DA84202D1042510E037E07E
:10040000264DA84201D105250AE0254DA84201D17B
:10041000062505E0234DA84201D1072500E0082567
:10042000BD402543C6F80858DBF800405D464E68DD
:100430009C43F60300D51C432C60DEF80040754653
:100440004E689C43B60300D51C432C600B4D083509
:100450002C684E689C43F60200D51C432C60074D67
:100460000C352C684E689C43B60200D51C432C60AA
:10047000521C102AFFF44EAFBDE8F88F003C01403B
:1004800044380240003001400000024000040240B5
:1004900000080240000C024000100240001402401C
:1004A00000180240001C02400AB181617047090433
:1004B000FBE700000148806870470000240000202E
:1004C000024881680278114481607047240000204E
:1004D0000B4810B5016841F400710160016841F4F6
:1004E00080610160016841F480710160032000F0C7
:1004F0006FF8002000F006F800F024F8002010BD8E
:10050000003C024070B50D4D04464FF47A712878D6
:10051000B1FBF0F00A490968B1FBF0F000F0E2FA33
:1005200048B9102C07D200222146501E00F030F8A6
:1005300000206C6070BD012070BD00002400002010
:10054000300000200A4808B5016841F4804101608C
:10055000006800F4804000900548001F016841F0E9
:1005600080510160006800F08050009008BD0000DC
:1005700044380240002809DB00F01F0201219140AD
:100580004009800000F1E020C0F800117047000031
:10059000F0B40E4B1B680C46C3F30223C3F10705EE
:1005A000042D00D90425191D072901D2002300E0DC
:1005B000DB1E012606FA05F1491E214099409E40A6
:1005C000761E16403143F0BC01F005B80CED00E09A
:1005D000064900F0070208684FF6FF03184040EA9A
:1005E0000220034A10430860704700000CED00E051
:1005F0000000FA052DE9F0470E46050065D0DFF84A
:100600001481D8F80000F7B200F00F00B04207D212
:1006100088F80070D8F8000000F00F00B04254D104
:1006200028683D4C810712D5400703D5206840F467
:10063000E05020602878000703D5206840F460402F
:1006400020602068A96820F0F00008432060287826
:10065000C0072DD0304968680839012812D0022817
:1006600013D0032811D00968890700292DDA2168E1
:1006700021F0030101432160FFF71CFF814641F295
:10068000883A0EE009688903EFE709688901ECE719
:10069000FFF710FFA0EB0901514502D90320BDE887
:1006A000F0872068696800F00C00B0EB810FEFD193
:1006B000D8F80010404601F00F01B14207D9077089
:1006C000006800F00F00B04201D00120E7E7287871
:1006D000400705D52068E96820F4E0500843206011
:1006E0002878000706D52068296920F4604040EA90
:1006F000C100206000F036F82168084AC1F30311F8
:10070000515CC840064908600020FFF7FBFE00204E
:10071000C5E70000003C024008380240B41600085B
:10072000300000200448054900680968044AC1F304
:100730008221515CC84070473000002008380240D8
:10074000C41600080448054900680968044AC1F352
:100750004231515CC84070473000002008380240E8
:10076000C4160008154810B5006810F00C021448B3
:1007700013D01449042A0FD0082A0ED10F4C241F7D
:100780002268236802F03F025B0207D52068C0F3AD
:100790008810A0FB010106E0084610BD2168C1F3E6
:1007A0008811A1FB00010023FFF70AFD2168C1F3B6
:1007B0000141491C4900B0FBF1F010BD083802406E
:1007C0000024F40040787D012DE9F84F050076D033
:1007D0002878DFF8F8B2BE4CC00749D0DBF800102B
:1007E0005846C1F38101012908D00068C0F3810097
:1007F00002280AD1201D0068400206D52068800327
:1008000036D568680028E2D032E06868B0F5803FED
:1008100010D0B0F5A02F206810D020F480302060D8
:10082000206820F4802020606868A0B1FFF742FEB5
:1008300006460CE0206840F48030F4E740F4802065
:100840002060F7E7FFF736FE801B642873D8206826
:100850008003F7D50CE0FFF72DFE064605E000BF4C
:10086000FFF728FE801B6428F0D820688003F7D4A7
:100870002878DFF8608280074FF000093ED5DBF86A
:100880000010584611F00C0F09D00068C0F3810029
:1008900002280BD18D48001F0068400206D4206852
:1008A000800715D5E868012809D111E0E868B8B1DA
:1008B0000120C8F80000FFF7FDFD064605E002E153
:1008C000FFF7F8FD801B0228C0D820688007F7D505
:1008D0002068296920F0F80040EAC10020600DE09E
:1008E000C8F80090FFF7E6FD064604E0FFF7E2FDDA
:1008F000801B02281FD820688007F7D428780007BB
:1009000022D5724E744869696C3671B1012101605B
:10091000FFF7D0FD074604E0FFF7CCFDC01B02281F
:1009200009D830688007F7D50EE0C0F80090FFF7CF
:10093000C1FD074605E083E0FFF7BCFDC01B0228B0
:100940007ED830688007F7D42878400768D5DFF86C
:100950007CA100270AF1380ADAF80000C0000BD4A5
:10096000DAF8001041F08051CAF80010DAF80000FF
:10097000012700F080500090584E3068C00510D418
:10098000306840F480703060FFF794FD009005E01F
:10099000FFF790FD0099401A022851D83068C00531
:1009A000F6D54A4EA868683601280FD00528306869
:1009B00010D020F001003060306820F0040030607A
:1009C000A868B8B1FFF776FD00900FE0306840F0FE
:1009D0000100F4E740F004003060F7E7FFF76AFD3C
:1009E0000099411A41F28830814264D8306880070A
:1009F000F4D50EE0FFF75EFD009007E0FFF75AFD2B
:100A00000099411A41F28830814254D830688007F9
:100A1000F4D42FB1DAF8001021F08051CAF8001098
:100A2000A869C0B3DBF80010C1F3810102294AD0E4
:100A30000228484607D0C8F86000FFF73BFD00E0F9
:100A400039E005463AE04746C8F86000FFF732FD56
:100A5000064604E0FFF72EFD801B02282BD82068F5
:100A60008001F7D4D5E907010843A96A1C4A49085F
:100A700002EB01416A6A41EA8211084395F82C10A1
:100A800040EA01611148001F016001203866FFF74C
:100A900011FD054605E014E0FFF70CFD401B0228A0
:100AA00009D820688001F7D50BE000BFFFF702FDF1
:100AB000401B022802D90320BDE8F88F206880017E
:100AC000F4D40020F8E70120F6E7000008380240DF
:100AD0000038024000004742800E4742007000404C
:100AE0000000FFFF10B5401EB0F1807F01D3012050
:100AF00010BD4FF0E02460610F21601700F06BFD26
:100B00000020A06107202061002010BD7047000078
:100B100070B5026804461068D168536910F00F0F71
:100B200050D003F0010501F4907635435DD0C20743
:100B300005D0CA0503D5E26B42F00102E263420729
:100B400005D5DA0703D0E26B42F00202E2638207C6
:100B500005D5DA0703D0E26B42F00402E263020734
:100B600005D5DA0703D0E26B42F00802E263E26BDC
:100B7000002A33D0800604D5880602D5204600F02E
:100B800017FB20684069E16BC0F38010090700D4AF
:100B900028B3204600F0FEFA2068416949061AD5BC
:100BA000416921F040014161606BA0B11B490165C1
:100BB000606BFFF77CFB002810D0606B016DBDE817
:100BC00070400847830610D58B060ED52046BDE839
:100BD000704000F0EDBA2046FFF798FF70BD204648
:100BE000FFF794FF0020E06370BD030606D50B06F7
:100BF00004D52046BDE8704000F07CBC4006F3D52B
:100C00004806F1D5D168204621F04001D16020216D
:100C100084F8391000F0B1F970BD000085110008AA
:100C200070B5040004D094F83900002510B106E036
:100C3000012070BD84F83850204600F023F82420AD
:100C400084F839002068C16821F40051C160204651
:100C500000F0FAFA2068016921F4904101612068EE
:100C6000416921F02A0141612068C16841F40051C5
:100C7000C160E563202084F8390084F83A00002040
:100C800070BD0000F0B587B0044614216846FFF738
:100C9000CFFA3A48384E25683849103802220123E5
:100CA0000324B5421FD10D6845F400250D60096885
:100CB00001F400210591016841F004010160006820
:100CC000694600F004000590A0028DE81D00082090
:100CD00004902B48FFF710FB002211463420FFF749
:100CE00057FC342022E0274F0726BD4222D123495A
:100CF000091D0D6845F010050D60096801F010012F
:100D00000591016841F0020101600068694600F048
:100D100002000590C0208DE85D001B48FFF7ECFA4B
:100D2000002211462520FFF733FC2520FFF722FC87
:100D300007B0F0BD154FBD42FAD10D6845F400353E
:100D40000D60096801F400310591016841F0080166
:100D500001600068694600F00800059060208DE899
:100D60005D000B48FFF7C8FA002211462620FFF766
:100D70000FFC2620DAE70000004C0040403802401B
:100D800000080240001001400004024000440040FE
:100D9000000C024090F83A30202B22D1F9B1F2B188
:100DA00090F83830012B1CD081628285C2850021E9
:100DB000C163222280F83A2080F838100168CA689E
:100DC00042F48072CA6001684A6942F001024A61D5
:100DD0000068C16841F02001C16000207047012017
:100DE00070470220704700002DE9F04100682D494E
:100DF0002D4F012607F1110488421CD12078E8BB51
:100E00000A230522F91D294800F05AF8F81D851F0C
:100E10004178297081786970C078A8700A2303220C
:100E20002946224800F04CF8A878012800D13E70ED
:100E30002670BDE8F0811E49884220D16078E8B96B
:100E400019490A2305220C31184800F039F81648D0
:100E50000A230C30A0F10805417829708178697067
:100E6000C078A87003222946104800F029F8A87815
:100E7000012801D1022038706670DAE702E00D49DE
:100E80008842D6D10849322307221D310A4800F092
:100E900017F8BDE8F0410449322307221D31074805
:100EA00000F00EB8001001400000002034000020C7
:100EB00000440040004C004074000020B4000020BA
:100EC0002DE9F843044690F839001F4616460D46B2
:100ED000202850D1A5B19EB194F8380001284AD0FD
:100EE000012084F838004FF00008C4F83C8021202D
:100EF00084F83900FFF7DEFAA6848146E68426E00E
:100F00000120BDE8F883E08C401EE084A0684B46D9
:100F1000B0F5805F4FF000024FF08001204600974F
:100F200003D000F018FBE8B90DE000F014FBC8B9DD
:100F300028882168C0F308004860206908B16D1C4A
:100F400005E0AD1C03E0216815F8010B4860E08C5A
:100F50000028D8D14B46002240212046009700F0BF
:100F6000FAFA08B10320CCE7202084F8390084F88D
:100F700038800020C5E70220C3E77047FEE7000085
:100F800070B586B014216846FFF752F91648002460
:100F9000016841F008010160016801F00801059154
:100FA000016841F004010160016801F0040105914C
:100FB000016841F00201016000680C4E00F002007F
:100FC0004FF470450590002229463046FFF76CFA31
:100FD00001200095CDE90104694630460394FFF7EE
:100FE0008BF906B070BD000030380240000C0240A2
:100FF0000C4810B50A4901604FF4E131416000210D
:1010000081600C22C160C0E904128161C161FFF7F7
:1010100007FE002803D0BDE81040FFF747B910BD18
:10102000004C0040340000200C4810B50A49016013
:101030004FF4E1314160002181600C22C160C0E9C0
:1010400004128161C161FFF7EBFD002803D0BDE808
:101050001040FFF72BB910BD0010014074000020B4
:101060000C4810B50A4901604FF4E131416000219C
:1010700081600C22C160C0E904128161C161FFF787
:10108000CFFD002803D0BDE81040FFF70FB910BD19
:1010900000440040B4000020FEE7704770477047EE
:1010A000FFF70EBA30B593B030216846FFF7C0F8AD
:1010B00014210CA8FFF7BCF818480025016841F07E
:1010C00080510160006800F0805011901448016860
:1010D00041F4804101600068022400F480401190D6
:1010E0000120039010200490009406940820CDE97C
:1010F00007504820CDE9090403200B906846FFF70C
:1011000063FB0CA90F2081E83100E002CDE90F0557
:1011100002210CA8FFF76EFA13B030BD4038024030
:10112000007000401048016841F4700101600F48F0
:10113000016841F0010101600C4A00210832116090
:1011400002680B4B1A400260031D0A4A1A600268CB
:1011500022F48022026005480C30016002495806E2
:10116000803908607047000088ED00E000380240D8
:10117000FFFFF6FE103000240148FFF7C9BC000055
:101180003400002010B5806B0021C185C184FFF7B9
:10119000BDFC10BD0168CA6822F49072CA60016883
:1011A0004A6922F001024A61202180F83A10704712
:1011B00010B590F83A10222901D0022010BD8168A4
:1011C000B1F5805F11D00169002901681FD049681D
:1011D00001F07F03816A4A1C82620B70C18D491E37
:1011E0000904090CC18518D02BE00269816A002A24
:1011F0000268526805D0D2B20A80816A491C8162B5
:10120000ECE7C2F308020A80816A891CF7E74A68A2
:10121000816A4B1C83620A70E0E70168CA6822F0A9
:101220002002CA600168CA6822F48072CA6001683C
:101230004A6922F001024A61202180F83A10FFF742
:10124000D3FD002010BD00002DE9F04104460068E8
:101250000169E26821F44051114301612169A068EC
:10126000E26908436169114322680843D16849F281
:101270000C6399430143D16020684169A26921F45C
:10128000407111434161E2696425B2F5004F97480E
:10129000974922684FF032083FD08A4201D08242FB
:1012A0007CD1FFF74FFA00EBC00101EB0010616841
:1012B0008900B0FBF1F6FFF745FA00EBC00101EB46
:1012C000001061688900B0FBF1F0B0FBF5F06FF041
:1012D0001801484306EB800108EB0110B0FBF5F064
:1012E00000F0F006FFF72EFA00EBC00101EB001052
:1012F00061688900B0FBF1F0B0FBF5F006EB001679
:10130000FFF720FA00EBC00101EB001061688900D3
:10131000B0FBF1F7FFF716FAD2E08A4201D0824221
:101320003DD1FFF70FFA00EBC00101EB001061683F
:101330004900B0FBF1F0B0FBF5F00601FFF702FA4F
:1013400000EBC00101EB001061684900B0FBF1F750
:10135000FFF7F8F900EBC00101EB001061684900EC
:10136000B0FBF1F0B0FBF5F06FF01801484307EB6C
:10137000800108EBC100B0FBF5F000F0F80006EBCF
:101380004006FFF7DFF900EBC00101EB00106168D8
:101390004900B0FBF1F7FFF7D5F93CE055E0FFF766
:1013A000C1F900EBC00101EB001061684900B0FB1E
:1013B000F1F0B0FBF5F00601FFF7B4F900EBC00166
:1013C00001EB001061684900B0FBF1F7FFF7AAF9E3
:1013D00000EBC00101EB001061684900B0FBF1F0C7
:1013E000B0FBF5F06FF01801484307EB800108EB04
:1013F000C100B0FBF5F000F0F80006EB4006FFF787
:1014000091F900EBC00101EB001061684900B0FBED
:10141000F1F7FFF787F900EBC00101EB00106168FD
:101420004900B0FBF1F0B0FBF5F06FF01801484354
:1014300007EB800108EBC100B0FBF5F000F00700FE
:10144000216830448860BDE8F081FFF76BF900EB5C
:10145000C00101EB001061688900B0FBF1F6FFF7F5
:1014600061F900EBC00101EB001061688900B0FB7D
:10147000F1F0B0FBF5F06FF01801484306EB800186
:1014800008EB0110B0FBF5F000F0F006FFF74AF9A9
:1014900000EBC00101EB001061688900B0FBF1F0C6
:1014A000B0FBF5F006EB0016FFF73CF900EBC001CE
:1014B00001EB001061688900B0FBF1F7FFF732F92A
:1014C00000EBC00101EB001061688900B0FBF1F096
:1014D000B0FBF5F06FF01801484307EB800108EB13
:1014E0000110B0FBF5F000F00F00A9E70014014077
:1014F0000010014090F83910212901D002207047D6
:101500008168B1F5805F016A0BD04A1C02620268F3
:1015100009785160C18C491E0904090CC1840ED0A0
:1015200017E009880268C1F30801516001690029C8
:10153000016A02D0491C0162ECE7891CFBE70168E3
:10154000CA6822F08002CA600068C16841F04001A8
:10155000C160002070472DE9F041984617460E46BD
:101560000446069D1DE0681C1BD02DB1FEF7A2FFAE
:10157000A0EB0800A84214D92068C16821F4D071FA
:10158000C1602068416921F001014161202084F897
:10159000390084F83A00002084F838000320BDE8C0
:1015A000F0812068006836EA000004D00020B842CC
:1015B000D9D00020F3E70120F9E700000148FFF748
:1015C000A7BA0000740000200148FFF7A1BA00008C
:1015D000B4000020FEE70907090E002804DB00F133
:1015E000E02080F80014704700F00F0000F1E020C8
:1015F00080F8141D704702E008C8121F08C1002AB5
:10160000FAD170477047002001E001C1121F002A83
:10161000FBD17047FEF75CFFFFF744FDFFF7B0FC1E
:10162000FFF71EFDFFF7E4FCFFF7FEFC3223072265
:101630001C491D48FFF744FC1A4905220F391A4876
:10164000FFF7A8FB6420FEF745FE32230722154969
:101650001648FFF735FC134905220A391348FFF7EE
:1016600099FB104C163C2078012805D10D49072222
:10167000C91D0F48FFF78EFB2078022805D10949C4
:101680000722C91D0948FFF785FB064905220F39C6
:101690000548FFF77FFB034905220A390348FFF796
:1016A00079FBE0E71600002074000020B400002061
:1016B00034000020000000000000000001020304CC
:1016C000060708090000000001020304EC160008E8
:1016D0000000002034000000F61500082017000864
:1016E00034000020C440000006160008000000007E
:1016F00000000000000000000000000000000000EA
:101700000000FFFF000000000DFFFF000000000DC3
:101710000100000010000000000000000024F400A0
:040000050800018965
:00000001FF
